:10000300750B00750A00750940750840750F00757A
:100013000E00750D80750C40750B00750A0075098F
:1000230040750840750F00750E00750D80750C4006
:10003300AF0BAE0AAD09AC08A804A905AA06AB0725
:100043001201A78F138E128D118C101202AD8F80A7
:10005300AF0FAE0EAD0DAC0CA804A905AA06AB07F5
:100063001201A78F178E168D158C141202AD8F9067
:10007300AF17AE16AD15AC14AB13AA12A911A81085
:100083001200B68F1B8E1A8D198C181202AD8FA019
:10009300AF1BAE1AAD19AC181203DB8F1F8E1E8D6A
:0C00A3001D8C1C1202AD8FB002001B224D
:1000AF00020319E86480F8E933E83360110460F063
:1000BF00ED33EC337009E8FCE9FDEAFEEBFF2204B7
:1000CF0060DED3EB9FEA9EE99DE8C2E78CF0C2F7B2
:1000DF0095F0400CE8CCF8E9CDF9EACEFAEBCFFB7E
:1000EF001202E485D0F05804700320D5B3E80470F1
:1000FF00075002B2D502032392D5EC0460F7E4CC8B
:10010F00C0E0C398F8603B94186008400DD0E0FB46
:10011F000202FBE4FBFAC9FC8028E830E406E4C9DC
:10012F00FBE4CAFCE830E305E4C9CACBFCE854079A
:10013F006010F8C3E913F9EA13FAEB13FBEC13FCA5
:10014F00D8F130F52FC3E49CFCEF9BFFEE9AFEED48
:10015F0099FDD0E0FBEF4E4D4C701222DB030203F2
:10016F0020EC2CFCEF33FFEE33FEED33FDED30E7EB
:10017F00EB0202FBEF2BFFEE3AFEED39FDD0E0FB79
:10018F0050130BBB0003020323ED13FDEE13FEEF21
:08019F0013FFEC13FC0202FB4C
:1001A700EC4D6011E8497017ED33EC3304600DE452
:1001B700FCFFFEFD22E933E8330470F8020319124D
:1001C70002E458046009E4CC24815006285009024F
:1001D7000323284003020320C0E0EB4A7044B980A0
:1001E70006D0E0FB02030FEF4E701CBD8008EBFF4B
:1001F700EAFEE9FD80EBE98DF0A4FEE5F00202904E
:10020700E9CDF9EAFEEBFFEF89F0A4FCE5F0CE8932
:10021700F0A42EFFE435F0CD89F0A42DFEE435F0EF
:100227008067EF4E7005BD80D780C3EF8BF0A4AC1D
:10023700F0EE8BF0A42CFCE435F0F8EF8AF0A42C58
:10024700E5F038FCE433CB8DF0A42CFCE5F03BF86B
:10025700EE8AF0A42CFCE5F038F8E433CF89F0A45B
:100267002CFCE5F038CF3400CE89F0A42FFFE5F061
:100277003EFEE433C98DF0A42EFEE5F039CD8AF0B9
:10028700A42FFFE5F03EFEE43DFD33D0E0FB500731
:100297000BBB000F020323EC2CFCEF33FFEE33FE06
:0602A700ED33FD0202FB35
:1002AD00EDD2E7CD33EC3392D524814006E4FFFE49
:1002BD00FDFC22FCE4CFCECDCC24E0501174FF80A8
:1002CD00EDC3CC13CCCD13CDCE13CECF13CF047045
:0702DD00F030D5DE0203C979
:1003D70002031922EDA2E7D2E7F9EC3340F260F30A
:1003E700B4FF08ED547F70E8020323F82481C2E0CC
:1003F700C0E0F40428FAC313FCED92E7FD8C208DCE
:10040700218E228F23EEA2E7E9BA7F02C3133400BD
:100417009400FA75F091A4E5F013F494FE8AF0A421
:1004270033E5F033248CD313FDE492E7FE7F007CA1
:100437003F758302ECC0E0F8EDC0E0F9EEC0E0FAEA
:10044700EFC0E0FBAC20AD21AE22AF23120330D0CA
:10045700E0FBD0E0FAD0E0F9D0E0F81200B6ED64A6
:1004670080FD30E7011CD583CBED33CC33F8D0E0EA
:0A047700A2E71328C313CC13FD22E3
:1002E400E9D2E7C933E833F892D5EDD2E7CD33EC60
:0702F40033FC5002B2D522D9
:1002FB00EC30E7100FBF000C0EBE00080DBD000464
:10030B000BEB6014A2D5EB13FCED92E7FD2274FF0F
:10031B00FCFDFEFF22E480F8A2D574FF13FC7D8068
:02032B0080F060
:10032D00020323EC5D046005E85904700302031910
:10033D001202E4580460F6EC4860F2EC7004FDFE25
:10034D00FF22C82481C85007C39850060203209885
:10035D0050CEF582E9294B4A7005AB8202030F7529
:10036D00F0007C1A7880C3EF9BEE9AED99400DC397
:10037D00EF9BFFEE9AFEED99FDE842F0DC23ACF029
:10038D00D0E0FFD0E0FED0E0FDAB8220E7101BEB0C
:10039D0060BAEC2CFCEF33FFEE33FEED33FD0202C1
:1003AD00FBE803F830E705C0F075F000EF2FFFEE26
:0C03BD0033FEED33FD40B830E7C280AAEB
:0300000002048176
:0C048100787FE4F6D8FD758123020003AB
:0E03C900C3E49FFFE49EFEE49DFDE49CFC2245
:00000001FF
